:020000040000FA
:1000000058281920B400152020082104031953286A
:100010004D2084133408800664000E280F28A00A9F
:100020000319A10F0C2880065328FF3A8417800576
:100030005328A8000630A8190730840000308A0031
:100040002808073982070134023404340834103494
:10005000203440348034A301A200FF30A207031CE7
:10006000A307031C53280330A100DF3039202D28BB
:10007000A101E83EA000A109FC30031C4228A00712
:1000800003183F28A0076400A10F3F282018482824
:10009000A01C4C2800004C280800A009A109A00AB7
:1000A0000319A10A080083130313831264000800D4
:1000B000831686018312B8016400973038028A11D2
:1000C0000A12031877286430A000A10100308A01C9
:1000D0000120C830A000A10101308A0101200F30A9
:1000E0008A012B20B80A8A110A12031D5C28643089
:1000F0008A012B20B8016400793038028A110A1273
:1001000003189028C830A000A10101308A01012005
:100110000F308A012B20B80A8A110A12031D7B288E
:0A01200064308A012B208A015B285D
:02400E00753FFC
:00000001FF
